:100000000C9474010C9491010C9491010C94910145
:100010000C9491010C9491010C9491010C94910118
:100020000C9491010C9491010C9491010C94910108
:100030000C9491010C9491010C9491010C949101F8
:100040000C9491010C9491010C9491010C949101E8
:100050000C9491010C94C2060C9491010C949101A2
:100060000C9491010C949101808183848687898A04
:100070008C8E8F9192949597989A9B9D9EA0A2A307
:10008000A5A6A7A9AAACADAFB0B2B3B5B6B7B9BA79
:10009000BCBDBEC0C1C2C4C5C6C8C9CACBCDCECF07
:1000A000D0D2D3D4D5D6D7D9DADBDCDDDEDFE0E1C0
:1000B000E2E3E4E5E6E7E8E9EAEAEBECEDEEEEEFB1
:1000C000F0F1F1F2F3F3F4F5F5F6F6F7F8F8F9F9E3
:1000D000FAFAFAFBFBFCFCFCFDFDFDFDFEFEFEFE5C
:1000E000FEFFFFFFFFFFFFFF0000891112239B327D
:1000F0002446AD573665BF74488CC19D5AAFD3BEF8
:100100006CCAE5DB7EE9F7F88110080193331A2207
:10011000A5562C47B7753E64C99C408DDBBF52AED7
:10012000EDDA64CBFFF976E802218B3010029913E7
:100130002667AF763444BD554AADC3BC588ED19FB7
:100140006EEBE7FA7CC8F5D983310A2091121803C7
:10015000A7772E66B5543C45CBBD42ACD99E508F97
:10016000EFFB66EAFDD874C904428D5316619F7097
:100170002004A9153227BB364CCEC5DF5EEDD7FC77
:100180006888E1997AABF3BA85520C4397711E6087
:10019000A1142805B3373A26CDDE44CFDFFD56EC57
:1001A000E9986089FBBB72AA06638F7214409D5167
:1001B0002225AB343006B9174EEFC7FE5CCCD5DD37
:1001C0006AA9E3B8788AF19B87730E6295501C4147
:1001D000A3352A24B1163807CFFF46EEDDDC54CD17
:1001E000EBB962A8F99A708B088481951AA793B627
:1001F0002CC2A5D33EE1B7F04008C919522BDB3A17
:10020000644EED5F766DFF7C899400859BB712A6E6
:10021000ADD224C3BFF136E0C1184809D33B5A2AF6
:10022000E55E6C4FF77D7E6C0AA583B418869197C6
:100230002EE3A7F23CC0B5D14229CB38500AD91BD6
:10024000666FEF7E744CFD5D8BB502A499961087A6
:10025000AFF326E2BDD034C1C3394A28D11A580BB6
:10026000E77F6E6EF55C7C4D0CC685D71EE597F476
:100270002880A1913AA3B3B2444ACD5B5669DF7896
:10028000600CE91D722FFB3E8DD604C79FF516E466
:10029000A9902081BBB332A2C55A4C4BD7795E6876
:1002A000E11C680DF33F7A2E0EE787F61CC495D546
:1002B0002AA1A3B03882B193466BCF7A5448DD5956
:1002C000622DEB3C700EF91F8FF706E69DD414C526
:1002D000ABB122A0B9923083C77B4E6AD5585C4936
:1002E000E33D6A2CF11E780F11241FBECFEFD8E03A
:1002F000DEBFCDBF11E0A0E0B1E0E2E3F6E102C075
:1003000005900D92A231B107D9F728E0A2E1B1E042
:1003100001C01D92AC33B207E1F70E94D6090C94DC
:10032000170B0C9400000C946A0878948CE294E00B
:100330000E94070343E951E06CE274E088E095E035
:100340000E9451078AEF94E00E94C5018AEF94E071
:100350009093390880933808909337088093360833
:10036000AC016CE274E088E095E00C945D0890913B
:10037000C00095FFFCCF8093C60008958091C00017
:1003800087FFFCCF8091C6000895CF93DF93CDB750
:10039000DEB72E970FB6F894DEBF0FBECDBFDC01DF
:1003A0009EE0FD01892F11928A95E9F71092C50010
:1003B00087E68093C400E0ECF0E080818D7F80834D
:1003C00086E08093C20088E18093C1009E012F5F88
:1003D0003F4FF90111929A95E9F783E08C8387EBFF
:1003E00091E09A8789878EEB91E09C878B878EE0DE
:1003F000F90101900D928A95E1F72E960FB6F894C7
:10040000DEBF0FBECDBFDF91CF910895811106C031
:100410008091C000881F8827881F089580E0089574
:100420008091C00087FF03C08091C60008958FEFC0
:1004300008950F931F93CF93DF93182FC0912C082B
:10044000D0912D08FE01E959FF4F8081811124C010
:1004500080E490E09E8F8D8F1C8E1B8E1A8E01E0A3
:100460000083299A2091090130910A0140910B01E2
:1004700050910C01A0EBB4E00E94170A6056704F37
:100480008F4F9F4F20E43FE140E050E00E94E6099B
:100490003B8B2A8B009313010FB7F8942091050131
:1004A000309106014091070150910801A0EBB4E0A2
:1004B0000E94170A6056704F8F4F9F4F20E43FE114
:1004C00040E050E00E94E6093D8B2C8B0FBFE0918D
:1004D0002C08F0912D085FB7F89423A134A1878DE3
:1004E00090A12817390739F425A136A181A192A13D
:1004F0002817390761F025A136A183A194A101979E
:1005000041E02817390709F040E0842F01C081E05D
:100510005FBF80FDDCCFE0912C08F0912D084FB734
:10052000F894A5A1B6A11C9325A136A181A192A101
:100530002817390719F4878D90A103C085A196A1CA
:10054000019696A385A34FBFDF91CF911F910F9185
:100550000895E0912C08F0912D084FB7F894EB58CE
:10056000FF4F24813581868197814FBF2817390736
:10057000E1F0E0912C08F0912D082FB7F894EB589A
:10058000FF4FA481B58182819381A817B90719F41F
:100590008081918104C0A481B581CD0101969583AC
:1005A00084838C912FBF90E008958FEF9FEF089583
:1005B00081E080931201089581E0809312011092EE
:1005C000800089E18093810081E896E09093870024
:1005D0008093860080911201882321F080E480932B
:1005E0007C0002C010927C003898409880917E0078
:1005F000816080937E0087E080937B008CEE809307
:100600007A008AB1886F8AB9219A229A08950F9345
:100610001F93CF93DF93CDB7DEB72E970FB6F89425
:10062000DEBF0FBECDBF8C018AECD8011D928A952A
:10063000E9F710932D0800932C0880E490E0F8016E
:10064000968F858FC80180599F4FE859FF4F91833E
:1006500080839783868395838483049693838283A0
:100660000996D801AB58BF4F11969C938E9317965D
:100670009C938E93169715969C938E931497CF9672
:1006800013969C938E93129785599109D801909651
:100690009C938E935F9796969C938E939597949642
:1006A0009C938E939397CF9692969C938E939197CB
:1006B00084E090E0A681B7811C9246815781228117
:1006C00033814217530719F42081318104C02681F8
:1006D00037812F5F3F4F378326830197009751F76C
:1006E0000E94DC022EE0FE013196DF01822F1D9276
:1006F0008A95E9F783E08C8389E192E09A8789877C
:1007000089EA92E09C878B87D80101900D922A9507
:10071000E1F72E960FB6F894DEBF0FBECDBFDF9186
:10072000CF911F910F9108950F931F93CF93DF9354
:100730008B01E0912C08F0912D0825A136A134A35E
:1007400023A3EC01080F191FC017D10721F08991CD
:100750000E941902F9CFDF91CF911F910F91089557
:10076000DC0156968C9156978111E9C058968C9170
:10077000589781119FC093962D913C91949795968F
:100780008D919C9196972817390739F454968D913D
:100790009C915597892B09F45CC059968C91599777
:1007A000811103C05A961C925A9781E059968C93F6
:1007B000599752968D919C915397009789F59396EE
:1007C0002D913C91949795968D919C919697281791
:1007D000390751F454968D919C91559701975596F0
:1007E0009C938E93549721C09396ED91FC9194978E
:1007F00091968D919C919297E817F90729F45F964D
:100800008D919C91909706C09396ED91FC91949751
:10081000CF01019694969C938E939397808106C006
:10082000019753969C938E9352978EE757968C938D
:10083000579757968C9157978B3191F593962D91A9
:100840003C91949795968D919C919697281739078E
:1008500041F410921301A959BF4F1C92299880E0CE
:1008600008959396ED91FC91949791968D919C911A
:100870009297E817F90729F45F968D919C919097CC
:1008800006C09396ED91FC919497CF0101969496B2
:100890009C938E939397808157968C93579706C01D
:1008A0008E57823018F459961C92599781E05896C9
:1008B0008C93589759962C9159975D968D919C9150
:1008C0005E972223A9F05A962C915A97253080F0F2
:1008D0005A961C925A978034910519F485E790E056
:1008E00002C080E490E05E969C938E935D9723C057
:1008F00058963C91589757962C915797232341F03F
:100900005A968C915A978F5F5A968C935A970FC02C
:100910005A961C925A978034910519F485E790E015
:1009200002C080E490E05E969C938E935D97330FB7
:1009300058963C93589788E056968C9356975D96B8
:10094000ED91FC915E975B968D919C915C97E80F81
:10095000F91F9F0131705C963C932E935B975696DE
:100960008C915697815056968C93FF27E038F1056D
:1009700030F08FEF90E0AC014E1B5F0BFA01E859AD
:10098000FF4F84912F3F310511F008F080950895B5
:10099000EF92FF920F931F93CF93DF93FC018C0193
:1009A00001541F4FD8014D915C91119712971196E8
:1009B0005C934E93A555B10914968D919C91159712
:1009C00012962D913C9113978217930721F42D9144
:1009D0003C91119707C014968D919C9115979C019D
:1009E0002F5F3F4F15963C932E931497EC0188810F
:1009F0008602C00111249595879595958795E80104
:100A0000998388837F01D3ECED0EF11CE7012881E7
:100A100039818F010F531F4FE80139832883840FD9
:100A2000951F35952795820F931FE701998388833A
:100A3000AF014B535F4F21E0181619060CF420E06C
:100A4000EA018881880F822B888316968D919C916C
:100A50001797EC01688316962D913C911797129683
:100A60008D919C9113972817390721F48D919C91B2
:100A7000119705C016968D919C9117970196179620
:100A80009C938E931697DA019C91892F8695869573
:100A900089278370DF01AA53BF4F833039F48C91CB
:100AA000803214F48F5F01C081508C938C91885FE9
:100AB0008C9380340CF45FC18F738C93DF01A95346
:100AC000BF4F8C91880F97702BEF290F233010F0B8
:100AD000933009F481608C939C91892F86958927A6
:100AE000809581709685990F892B86878E3709F0BE
:100AF0004EC0DF01AB58BF4F14962D913C91159716
:100B00008D919C9111972817390759F416962D91BC
:100B10003C91179712968D919C911397281739073E
:100B200081F016962D913C91179714968D919C917A
:100B30001597019741E02817390709F040E0842F05
:100B400001C081E080FDDCC01696CD91DC91179745
:100B50008EE7888316962D913C91179712968D916A
:100B60009C9113972817390721F48D919C91119727
:100B700005C016968D919C911797019617969C9398
:100B80008E93169781E0818B2A9A41E0BCC0982F02
:100B90009F779F3719F4118A2A98EDC0918999237C
:100BA00009F4E9C0982F9F739E3309F4E4C080FFD5
:100BB00003C080898068808B87858F5F8787908955
:100BC000883008F4A5C0DF01AB58BF4F82E8890F19
:100BD000823018F09B3109F04BC014962D913C9156
:100BE00015978D919C9111972817390759F41696EE
:100BF0002D913C91179712968D919C9113972817E0
:100C0000390781F016962D913C91179714968D9186
:100C10009C911597019741E02817390709F040E0AA
:100C2000842F01C081E080FD1FC01696CD91DC911C
:100C300017978BE1888316962D913C911797129602
:100C40008D919C9113972817390721F48D919C91D0
:100C5000119705C016968D919C911797019617963E
:100C60009C938E93169704C0118A2A9840E001C085
:100C700041E014962D913C9115978D919C9111977F
:100C80002817390759F416962D913C91179712960B
:100C90008D919C9113972817390781F016962D9105
:100CA0003C91179714968D919C911597019751E05F
:100CB0002817390709F050E0852F01C081E080FD39
:100CC0001FC080891696CD91DC9117978883169660
:100CD0002D913C91179712968D919C9113972817FF
:100CE000390721F48D919C91119705C016968D912D
:100CF0009C911797019617969C938E93169703C015
:100D0000118A2A9840E0108A1786442321F033C0C4
:100D10009695908B30C0DF01A853BF4F8D919C9169
:100D20001197816011969C938E93EB58FF4F24810D
:100D30003581808191812817390739F426813781DF
:100D4000828193812817390761F026813781848158
:100D50009581019741E02817390709F040E0842F79
:100D600001C081E080FF07C08681978195838483DD
:100D700011961C921E92DF91CF911F910F91FF90BF
:100D8000EF9008951F920F920FB60F9211242F9398
:100D90003F934F935F936F937F938F939F93AF9303
:100DA000BF93EF93FF9380E286BB609178007091D0
:100DB00079007695679576956795605880912C08AF
:100DC00090912D080E94C80480911301882349F056
:100DD00080912C0890912D080E94B003807F88603C
:100DE00001C080E88BB98091F6049091F704A0913E
:100DF000F804B091F9040196A11DB11D8093F60489
:100E00009093F704A093F804B093F904FF91EF9145
:100E1000BF91AF919F918F917F916F915F914F9112
:100E20003F912F910F900FBE0F901F901895FF923A
:100E30000F931F93CF93DF93EC01F62E82E8860F7A
:100E40008E01085E1C4F823018F08BE1681307C0DA
:100E5000F801608171818BE190E00E94BE0AFE0181
:100E6000E25EFC4F20813181F901EF25FF27EE0F73
:100E7000FF1FE851FF4F45915491C25EDC4F232F75
:100E800033272427352739832883F801608171812E
:100E90008F2D90E0DF91CF911F910F91FF900C94D7
:100EA000BE0A24E233E0DC01F9011D923197E9F733
:100EB000FC01E85EFC4F7183608338965183408368
:100EC00032972FEF3FEF3183208332973183208396
:100ED00008953F924F925F926F927F928F929F926E
:100EE000AF92BF92CF92DF92EF92FF920F931F9338
:100EF000CF93DF932C013C0128EE621A2CEF720A8B
:100F00006C014DEDC41A4CEFD40AEC01CE5DDC4F00
:100F10008C01065E1C4F7C0184EEE81A8CEFF80A07
:100F200033243394AA24AA94BA2C4201A0EE8A1A3C
:100F3000ACEF9A0AF301808191810E94800A8F3F71
:100F4000FFEF9F0709F458C0D6012C91211128C04A
:100F50008E379105D1F4F80180819181429768F034
:100F6000D7018D919C91883B904F39F4D401ED913C
:100F7000FC91309711F0C20109953882F701B182D6
:100F8000A082D8011D921C92D5CF8F37910511F404
:100F90001882D0CF8B31910519F4F6013082CACF77
:100FA0002881222331F1D8012D913C912831B3E0E1
:100FB0003B07F0F4A9014F5F5F4FF8015183408375
:100FC000F201E20FF31F8083D7012D913C91F901CB
:100FD000E827FF27EE0FFF1FE851FF4F85919491FF
:100FE000232F332728273927F7013183208301C096
:100FF0001882D6011C929ECFDF91CF911F910F9145
:10100000FF90EF90DF90CF90BF90AF909F908F9028
:101010007F906F905F904F903F9008958F929F9236
:10102000AF92BF92CF92DF92EF92FF920F931F93F6
:10103000CF93DF938C014B016A017C0182EEE81AA9
:101040008CEFF80A8FEF9FEFF701918380835801AF
:10105000F8EEAF1AFCEFBF0AF501608171818EE7EF
:1010600090E00E94BE0AE401C80CD91CCC15DD0535
:1010700029F06991C8010E941707F8CFF701608134
:10108000C1816095C8010E9417076C2F6095C80147
:101090000E941707F501608171818EE790E0DF9172
:1010A000CF911F910F91FF90EF90DF90CF90BF9065
:1010B000AF909F908F900C94BE0A909330088093CD
:1010C0002F085093FB044093FA0470933208609306
:1010D00031080895EF92FF920F931F93CF93DF9300
:1010E000EC016091FA047091FB0480EC90E00E94A6
:1010F000BE0A6091FA047091FB0480E090E00E94C7
:10110000BE0A8E017E0186EEE81A8CEFF80AF7011E
:101110008081918102976091FA047091FB0498019B
:101120002C1B3D0B2817390708F5F80181918F0119
:10113000803C59F48BED90E00E94BE0A6091FA0465
:101140007091FB048CED90E00EC08B3D59F48BED5B
:1011500090E00E94BE0A6091FA047091FB048DED4C
:1011600090E001C090E00E94BE0AD1CF80EC90E0F8
:10117000DF91CF911F910F91FF90EF900C94BE0AD9
:101180008F929F92AF92BF92CF92DF92EF92FF9297
:101190000F931F93CF93DF93EC017B016A01E091E2
:1011A0003108F09132088189811143C00E94700A90
:1011B00090910001891788F4A601B701CE01DF9153
:1011C000CF911F910F91FF90EF90DF90CF90BF9044
:1011D000AF909F908F900C940E088FB7F8948090EA
:1011E000F6049090F704A090F804B090F9048FBF33
:1011F00020910101309102014091030150910401BD
:10120000AAE0B0E00E94170A4FB7F8940091F604E4
:101210001091F7042091F8043091F9044FBF081998
:1012200019092A093B09061717072807390764F324
:10123000B6CFE0913108F09132088189882309F412
:10124000AECF80912F08909130080E946907E091FD
:101250003108F0913208E853FF4F80819181892B4A
:1012600041F311821082DF91CF911F910F91FF9076
:10127000EF90DF90CF90BF90AF909F908F900895A8
:10128000282F809133088823A1F0203C01F580911C
:101290000D01811111C01092330840913408509112
:1012A000350864E171E080912F08909130080C942A
:1012B000C008203C09F079C081E0809333088EEFAC
:1012C00080930D0110923508109234080895809192
:1012D000340890913508883133E0930708F065C0F1
:1012E00030910D01009731F43E3F21F42F7020938F
:1012F0000D01089531111FC02B3D21F481E0809331
:101300002E08089530912E08332349F02C3D21F00A
:101310002D3D19F42BED01C020EC10922E08AC01EC
:101320004F5F5F4F5093350840933408FC01EC5EEB
:10133000FE4F20830895313071F430E0AAE0B0E030
:101340000E94080A6093090170930A0180930B01BF
:1013500090930C010895343089F43AE0239FC00142
:101360001124AA2797FDA095BA2F80930501909389
:101370000601A0930701B09308010895333089F462
:101380003AE0239FC0011124AA2797FDA095BA2F08
:101390008093010190930201A0930301B093040193
:1013A0000895323011F42093000108950E949501B0
:1013B00088E095E00E94690780E00E940602882389
:1013C000B9F30E9410020E944009F2CFA1E21A2E46
:1013D000AA1BBB1BFD010DC0AA1FBB1FEE1FFF1FD9
:1013E000A217B307E407F50720F0A21BB30BE40B29
:1013F000F50B661F771F881F991F1A9469F7609570
:101400007095809590959B01AC01BD01CF01089529
:10141000A29FB001B39FC001A39F700D811D112435
:10142000911DB29F700D811D1124911D08950E9480
:10143000080AA59F900DB49F900DA49F800D911D4B
:10144000112408958F929F92AF92BF92CF92DF9214
:10145000EF92FF92CF93DF93EC01688179818A81CB
:101460009B81611571058105910521F464E279ED97
:101470008BE597E02DE133EF41E050E00E94F00A68
:1014800049015A019B01AC01A7EAB1E40E94170A85
:101490006B017C01ACEEB4EFA50194010E94120B2C
:1014A000C60ED71EE81EF91EF7FE06C081E0C81A58
:1014B000D108E10880E8F80AC882D982EA82FB8272
:1014C000C6019F77DF91CF91FF90EF90DF90CF9093
:1014D000BF90AF909F908F9008950E94220A089528
:1014E0008EE091E00E94220A0895A0E0B0E080938F
:1014F0000E0190930F01A0931001B0931101089574
:10150000CF93DF93EC012B8120FF33C026FF0AC06D
:101510002F7B2B838E819F8101969F838E838A816F
:1015200090E029C022FF0FC0E881F98180819927CE
:1015300087FD9095009719F420622B831AC031968D
:10154000F983E8830EC0EA85FB85099597FF09C0FA
:101550002B81019611F480E101C080E2822B8B8304
:1015600008C02E813F812F5F3F4F3F832E839927F5
:1015700002C08FEF9FEFDF91CF9108950F931F93DC
:10158000CF93DF93182F092FEB018B8181FD03C0CF
:101590008FEF9FEF20C082FF10C04E815F812C81B2
:1015A0003D81421753077CF4E881F9819F012F5F49
:1015B0003F4F39832883108306C0E885F985812F42
:1015C0000995892B29F72E813F812F5F3F4F3F835C
:1015D0002E83812F902FDF91CF911F910F9108952E
:1015E000052E97FB1EF400940E94070B57FD07D0B1
:1015F0000E94E60907FC03D04EF40C94070B5095AB
:101600004095309521953F4F4F4F5F4F08959095EE
:101610008095709561957F4F8F4F9F4F0895B7FFCD
:101620000C94170A0E94170A821B930B0895F894D2
:02163000FFCFEA
:101632003FC80000003200000096000000FE0100DA
:021642000000A6
:00000001FF
